:10000000B4019C29A4003808840036081021841308
:1000100000052C1C3606031920282408031D182867
:100020002A08FF3E031C21280A3024212A082128FF
:10003000240AFF3003192028240B20282B0821280C
:10004000AD09AD0C9729B416B41EB41234192D287D
:10005000FE39B500341503109729341A3528A60047
:1000600034164C2003183A282608532003183A283F
:10007000B41E972945206A2034113412B41138086F
:1000800084003608841780044B2838088400360919
:1000900080058417800508003F206A2045206620DF
:1000A0003508B4190138A2000830A300A20D0318C6
:1000B0003F20031C45206A206620A30B56283F20C2
:1000C0006A203808840036080005FF3E390884009D
:1000D000370948283908840037088004841737090D
:1000E00080054B28A501A400B5172730A3001030C8
:1000F00085200330A300E8308520A30164308520EB
:10010000A3010A30852024089028A2002508A10018
:100110002408A00060212008031DB513B51B0800AA
:10012000303E93280408A700861186108610831697
:100130008611861086100F30860583122708B418A2
:10014000BF283A30A100983032213330A600D320A6
:100150001330A10088303221D32064303121D320E4
:10016000643031212230A600D3202830BE200C304C
:10017000BE200630BE20B4142708BF283414A600C1
:10018000341CCD288610033C031CD228D220073013
:10019000A100D0303221031408003414FE3C0319AE
:1001A00097298614341C341086150F3086052608CE
:1001B000F03986048611A60E3418D3283230312146
:1001C00003140800B51329080319B5170530A80052
:1001D0002730A3001030F8200330A300E830F820C7
:1001E000A3016430F820A3010A30F8202408FF2876
:1001F000A2002508A1002408A00060212008A0007A
:10020000A8030319B513290803190929280203189B
:1002100008002008031DB513B51B0800303E9229C5
:1002200084178004972983169B001C141A089729A9
:1002300083169A001C1555309D00AA309D009C1411
:100240009C1820291C119729A301A200FF30A207A6
:10025000031CA307031C97290330A100DF303221C0
:100260002629A101E83EA000A109FC30031C3B297E
:10027000A00703183829A0076400A10F3829201807
:100280004129A01C4529000045290800A200023090
:100290005029A20006305029A301A20004305029A1
:1002A000A80023082102031D572922082002043038
:1002B00003180130031902302805031DFF30972968
:1002C000A501A4011030A600210DA40DA50D220842
:1002D000A4022308031C230FA50203187629220871
:1002E000A40723080318230FA5070310A00DA10DD1
:1002F000A60B6429200897291030A800A101A001AD
:10030000A70CA60C031C8A292208A007230803189F
:10031000230FA107A10CA00CA50CA40CA80B8029ED
:1003200024089729840031088A003008820083134A
:10033000031383126400080007309F00831605141E
:100340008514051505168515861006108312C23012
:10035000CA00C030C2002B30C3000230D1000130CF
:10036000C800C901D20164302421FE30932001303D
:100370009320203093205430932058309320203005
:1003800093204130932054309320563093202030D6
:100390009320353093202E309320373093204730F0
:1003A0009320483093207A30932020309320FE30E1
:1003B0009320C03093202A30932020309320763031
:1003C00093206530932072309320733093206930EE
:1003D00093206F3093206E30932020309320313063
:1003E00093202E30932031309320413093202030C1
:1003F00093202A3093200330A300E83025215208AF
:100400001321C40001305207B200B301B30D32080A
:100410001321C50042084407C00043080318013EE9
:100420004507C1000630B8000130B6000630B900FB
:100430000230B7004A082520410825204008252021
:100440008E302320F1222723643024210530B80088
:100450000830B600AC01FF30AA00AB010130AD009E
:100460004F080220CF000318862A0530B800083054
:10047000B6000130AC00FF30AA00AB010130AD0086
:1004800050080220D00003188B2A0530B800013034
:10049000B600AC010A30AA000230AB000130AD005A
:1004A0004B080220CB000318912A0530B800023017
:1004B000B600AC010A30AA000230AB000130AD003A
:1004C0004C080220CC000318A22A0530B8000430E2
:1004D000B600AC01FF30AA00AB010130AD004E0800
:1004E0000220CE000318AC2B0530B8001030B60047
:1004F000AC01FF30AA00AB010130AD004D08022075
:10050000CD000318C02A64302421262AD2014130AC
:10051000C600C701FF290230D2004230C600C70121
:10052000FF295108C4070318C50A4408A00045085C
:10053000A1000130A30090304921031DA12AC4016C
:10054000C5010A2A4408A0004508A100A301003003
:100550004621031DB82A4408A0004508A1005108FF
:100560004C21031DBD2A5108C402031CC5030A2ADD
:100570009030C4000130C5000A2AC401C5010A2A0E
:1005800064005108143C0319D62A640051080A3C3F
:100590000319EA2A64005108023C0319E32A6400A3
:1005A0005108013C0319DC2A2723262A0130D100F7
:1005B000C801C9012723262A0230D1000130C80012
:1005C000C9012723262A0A30D1000530C800C901F5
:1005D0002723262A1430D1000A30C800C901272356
:1005E000262A10304002B2002730031C013E41028F
:1005F000B3003208A6003308A7000430A200A3010C
:100600007C21BA002508BB003A08A0003B08A100E5
:100610000830A200A3016021BC002108BD003A08F7
:10062000A0003B08A1000830A200A301602124081B
:10063000B2002508B3007D30A600A7013208A20051
:100640003308A3007C21BE002508BF000800FE304F
:100650009320013093204630932052309320453030
:100660009320513093203A3093200530722003308C
:10067000A9003C08A4003D08A5009230B000B101DB
:10068000E2202E3093200330A9003E08A4003F084A
:10069000A5009230B000B101E2204D3093204830E7
:1006A00093207A309320203093204808A0004908F6
:1006B000A100A30100304621031D852BFE309320AD
:1006C000C030932056309320463093204F309320F3
:1006D0003A309320460893202030932020309320F6
:1006E0005030932061309320733093203A30932020
:1006F0004908A500480873204D30932048309320C6
:100700007A309320643024210800FE309320C030DA
:10071000932056309320463093204F3093203A3028
:10072000932046089320203093205030932061304E
:100730009320733093203A3093203530932030301B
:100740009320303093206B309320483093207A30C0
:100750009320643024210800520883169B008312E2
:100760004408182101305207B200B301B30D32081A
:1007700083169B00831245081821FE309320013018
:1007800093204630932052309320453093205130AF
:1007900093203A309320053072200330A9003C08A2
:1007A000A4003D08A5009230B000B101E2202E3037
:1007B00093200330A9003E08A4003F08A500923012
:1007C000B000B101E2204D309320483093207A30C0
:1007D000932020309320FE309320C03093204D3062
:1007E0009320453093204D3093204F30932052304A
:1007F000932049309320533093204530932020306C
:10080000932056309320463093204F3093203A3037
:100810009320460893200730A300D03025212723BA
:06082000262A6300112CE2
:02400E00653F0C
:08420000C8000000900001005D
:00000001FF
